:100000000C945A000C9477000C9477000C947700B1
:100010000C9477000C9477000C9477000C94770084
:100020000C9477000C9477000C9477000C94770074
:100030000C9477000C9477000C9477000C94770064
:100040000C94A5010C9477000C9477000C94770025
:100050000C9477000C9477000C9477000C94770044
:100060000C9477000C947700000024272A000025C8
:10007000282B000023262904040404040404040299
:100080000202020202030303030303010204081035
:100090002040800102040810200102040810200002
:1000A0000000070002010000030406000000000039
:1000B0000000000011241FBECFEFD4E0DEBFCDBF93
:1000C00011E0A0E0B1E0E0E4F7E002C005900D929D
:1000D000A231B107D9F711E0A2E1B1E001C01D9250
:1000E000AA31B107E1F70E949E010C949F030C9482
:1000F0000000EF92FF920F931F93CF93DF938091B5
:1001000000010E94E6028C01809102010E94E60239
:100110007C01809104010E94E602EC0180910601BD
:100120000E94E60260E070E0012B11F461E070E0F3
:1001300020E030E0892B11F421E030E0220F331F62
:1001400040E050E0CD2B11F441E050E0240F351F8A
:10015000220F331F40E050E0EF2811F441E050E05F
:10016000240F351F220F331FCB01820F931FDF9106
:10017000CF911F910F91FF90EF9008950E94790009
:10018000009749F460E070E080910E010E947402D3
:1001900060E070E047C08130910549F46FEF70E096
:1001A00080910E010E94740260EF70E03BC08230CB
:1001B000910549F46FEF70E080910E010E94740286
:1001C00060E170E02FC08330910579F467EF70E053
:1001D00080910E010E9474026CE170E080910C012C
:1001E0000E94740266EB70E023C08430910579F4BC
:1001F00067E170E080910E010E94740262E370E09A
:1002000080910C010E9474026FEF70E011C0853084
:10021000910599F463E370E080910E010E947402ED
:100220006CEF70E080910C010E94740260E070E05D
:1002300080910A010E94740208950F9791F46FEF64
:1002400070E080910E010E94740260EE70E0809177
:100250000C010E94740260EA70E080910A010E9421
:10026000740208950E94BE006AE070E080E090E0B1
:100270000E94E201089560E0809100010E94C8029E
:1002800060E0809102010E94C80260E08091040158
:100290000E94C80260E0809106010E94C80261E0ED
:1002A000809108010E94C80261E080910E010E94C5
:1002B000C80261E080910C010E94C80261E0809157
:1002C0000A010E94C8026FEF70E080910E010E9447
:1002D000740260EE70E080910C010E94740260EA8A
:1002E00070E080910A010E94740260ED77E080E086
:1002F00090E00E94E20160E070E080910E010E94B7
:10030000740260E070E080910C010E94740260E071
:1003100070E080910A010E94740261E080910801FE
:100320000E94320364E670E080E090E00E94E20107
:1003300060E0809108010E94320308950E9411023A
:100340000E943B010E943201FDCF1F920F920FB617
:100350000F9211248F939F93AF93BF9380911601B7
:1003600090911701A0911801B09119010196A11D5A
:10037000B11D8093160190931701A0931801B093BB
:100380001901BF91AF919F918F910F900FBE0F9068
:100390001F901895609116017091170180911801B6
:1003A0009091190127E0660F771F881F991F2A95E2
:1003B000D1F72DE730E040E050E00E947D03CA0114
:1003C000B9010895AF92BF92CF92DF92EF92FF9260
:1003D0000F931F935B016C010E94CA017B018C018A
:1003E0000E94CA016E197F09800B910B6A157B056B
:1003F0008C059D05A8F31F910F91FF90EF90DF9062
:10040000CF90BF90AF900895019751F0880F991F3A
:10041000880F991F02972FB7F8940197F1F72FBF14
:1004200008957894109216011092170110921801F5
:100430001092190184B5826084BD84B5816084BD49
:1004400085B5826085BD85B5816085BDEEE6F0E04D
:10045000808181608083E1E8F0E080818260808338
:10046000808181608083E0E8F0E08081816080832A
:10047000E1EBF0E0808184608083E0EBF0E080815C
:1004800081608083EAE7F0E08081846080838081FE
:1004900082608083808181608083808180688083A6
:1004A0001092C10008958093100108959091100159
:1004B0009295990F990F907C8F70982B90937C0058
:1004C00080917A00806480937A0080917A0086FD22
:1004D000FCCF20917800809179009927982F882768
:1004E0003327822B932B08951F93CF93DF93182FDD
:1004F000EB0161E00E94C802E12FFF27E156FF4FA8
:100500008491833051F480918000806880938000D2
:10051000D0938900C093880037C0843051F4809113
:100520008000806280938000D0938B00C0938A000B
:100530002BC0813029F484B5806884BDC7BD24C038
:10054000823029F484B5806284BDC8BD1DC0863068
:1005500041F48091B00080688093B000C093B300F4
:1005600013C0873041F48091B00080628093B00066
:10057000C093B40009C0C038D10514F460E001C0D4
:1005800061E0812F0E943203DF91CF911F91089586
:10059000282F3327C90185579F4FFC019491295873
:1005A0003F4FF9018491882381F0E82FFF27E85914
:1005B000FF4FE491FF27662329F4808190958923DA
:1005C000808308958081892B80830895482F552743
:1005D000CA0181569F4FFC012491CA0185579F4F44
:1005E000FC01949149585F4FFA013491332319F477
:1005F00080E090E00895222331F1233021F48091AE
:1006000080008F7705C0243031F4809180008F7D89
:100610008093800018C0213019F484B58F7704C00E
:10062000223021F484B58F7D84BD0DC0263021F4A5
:100630008091B0008F7705C0273029F48091B000F9
:100640008F7D8093B000E32FFF27EE58FF4FE4919A
:10065000FF27808120E030E0892311F021E030E0A5
:10066000C9010895482F5527CA0181569F4FFC01A3
:100670002491CA0185579F4FFC01949149585F4FBF
:10068000FA0134913323C1F1222331F1233021F4D3
:10069000809180008F7705C0243031F480918000F4
:1006A0008F7D8093800018C0213019F484B58F7736
:1006B00004C0223021F484B58F7D84BD0DC0263066
:1006C00021F48091B0008F7705C0273029F4809104
:1006D000B0008F7D8093B000E32FFF27E359FF4FD9
:1006E000E491FF27662329F48081909589238083F4
:1006F00008958081892B80830895A1E21A2EAA1B78
:10070000BB1BFD010DC0AA1FBB1FEE1FFF1FA217C1
:10071000B307E407F50720F0A21BB30BE40BF50BBE
:10072000661F771F881F991F1A9469F76095709547
:10073000809590959B01AC01BD01CF010895FFCF3D
:100740000200030004000500060009000A000B0077
:020750000100A6
:00000001FF
